:020000040000FA
:0600000060283D300130D4
:08000800A000030EA100831209
:100010008B1C2E288B1031181328B11C2E2864300D
:100020000102031C2D281428152816281728182823
:1000300019281A281B283110B114A810031005190B
:100040000314AA0DA90DA80DB00B2E2831152A08EE
:10005000AF002908AE002808AD00B11081010B11D6
:0A006000210E8300A00E200E0900FF
:1000C000203084008001840A60300402031C62280E
:1000D0001230B00076228316FF239000831283161D
:1000E0000C3085058701831285018701073099004F
:1000F0000030831691009F008312C8308316810060
:10010000831231309000003083168C00831210303F
:100110008B00BD1B8D28851DBF223D1BBE013D1BD5
:10012000BF013D1FB42281018E018F010B118B1085
:100130000B108C130C138C110C108B17AF20311972
:10014000C5204A22B30BAC28031085190314BA0D3D
:10015000F0303A020319A021BD18E7229E2864005E
:10016000311808000B1D08000B11B11031141230AA
:10017000B000051DC0283214831601138312080035
:1001800032108316011783120800321CCC282D0967
:100190000339AD00AE09AF09E4302F02F030031986
:1001A000AF004C302F020C300319AF006C302F021F
:1001B0003C300319AF00EC302F02FC300319AF00C4
:1001C000B3302F02F3300319AF001B302F020F3072
:1001D0000319AF003B302F023F300319AF00BB3093
:1001E0002F02FF300319AF0031110130B7008B131C
:1001F0002030370783169B001C141A088312A400B2
:10020000A50025101030370783169B001C141A0810
:100210008312A3000030370783169B001C141A08B2
:100220008312A2008B1722082D02031D9A2923088E
:100230002E06FC39031D9A29013003303702031DB5
:10024000452900302E060339031D2A29BF1F3329F3
:10025000BF13B11703302E060339031D3329BF1B0B
:100260003329BF17B11744302F065439031D3C29D9
:100270003F1F08003F13B11710302F065439031DDC
:1002800045293F1B08003F17B117AF13AF12AF113D
:10029000AF1024082F02031D712901303702031DFE
:1002A00056293E1856293E14B1178C2202303702C7
:1002B000031D5F29BE185F29BE14B1178E220330BB
:1002C0003702031D68293E1968293E15B11790228F
:1002D00004303702031D7129BE197129BE15B117EB
:1002E000942225082F02031D9A2901303702031D8D
:1002F0007E293E1C7E293E10B1179822023037021B
:10030000031D8729BE1C8729BE10B1179A2203300E
:100310003702031D90293E1D90293E11B1179C22E2
:1003200004303702031D9929BE1D9929BE11B1174A
:10033000A0229A29B70A0530370203180800F728C7
:10034000B601B3019630B4000130B5000130B700FA
:1003500085018701B1131A22AF20B30BD2290310F4
:1003600085190314BA0DF0303A0203190A2AB40BA6
:10037000D229013037020319A422023037020319AF
:10038000A822033037020319AC22043037020319C4
:10039000B0223708B6080319B6000319D029B603EE
:1003A0009630B400311DAC293111321CDC292D09E5
:1003B0000339AD00AE09AF0951302F065539031985
:1003C000F12905302F0655390319F12915302F066B
:1003D00055390319F12955302F0655390319F129DB
:1003E000AC29AF13AF12AF11AF108B13203037070A
:1003F000BC002F08BB00582210303707BC002E0865
:10040000BB00582200303707BC002D08BB00582223
:100410008B17142285018701B70AB6010530370210
:10042000031CAC29B4220800043037020319080069
:10043000850187016430B90033300F1E85000F1A23
:100440008501FF300F1A87000F1E8701AF20311D75
:100450001C2A3111321C312A2D090339AD00AE0995
:10046000AF0951302F06553903191A2A05302F06C6
:10047000553903191A2A15302F06553903191A2A26
:1004800055302F06553903191A2AB90B1C2A850134
:1004900087010800B11F0800B1131030BC003E08EE
:1004A000BB0058223030BC003F08BB005822080077
:1004B0003C088B1383169B001C141A0883128B179D
:1004C0003B02031908008B133B0883161C159A0086
:1004D0003C089B0055309D00AA309D009C14640090
:1004E0009C186F2A1C1183128B170800831600308A
:1004F0009B001C141A088312BD00831610309B0049
:100500001C141A088312BE00831630309B001C1482
:100510001A088312BF000800851608000516080097
:10052000BD18080085140800BD180800051408004F
:100530008512080005120800BD1808008510080083
:10054000BD180800051008000508203A85000800BD
:100550000508103A850008000508023A85000800E1
:100560000508013A850008003E188516BE180516D4
:10057000BD1808003E198514BE1905140800B601FF
:10058000B301B4013D1CC72A3D10BD14CA2AC030B6
:10059000BD053D143D083F39B6006400CF2AD02A7E
:1005A000D12AD22AD32A3330B41B8500B41F850147
:1005B000B30BCD2AB40BCD2A0310B60CB608031D1D
:1005C000CD2A0030BC003D08BB0058220800BF1FE8
:1005D000F22A3F1B85103F1B05143F1F85143F1F48
:0C05E00005100800851005100800080038
:084000000500000006000200AB
:02400E00CC01E3
:10420000010003000300030003000200020002009B
:10421000020000000000FF00FF00FF00FF00FF00A1
:10422000000000000000000000000000000000008E
:104230000000C000C000FF00FF00FF00FF00FF0003
:104240000100510005001500550051000500150042
:10425000550051000500FF00FF00FF00FF00FF00B8
:104260000000FF00FF00FF00FF00FF00FF00FF0055
:10427000FF00FF00FF00FF00FF00FF00FF00FF0046
:10428000FF00FF00FF00FF00FF00FF00FF00FF0036
:10429000FF00FF00FF00FF00FF00FF00FF00FF0026
:1042A000FF00FF00FF00FF00FF00FF00FF00FF0016
:1042B000FF00FF00FF00FF00FF00FF00FF00FF0006
:1042C000FF00FF00FF00FF00FF00FF00FF00FF00F6
:1042D000FF00FF00FF00FF00FF00FF00FF00FF00E6
:1042E000FF00FF00FF00FF00FF00FF00FF00FF00D6
:1042F000FF00FF00FF00FF00FF00FF00FF00AA001B
:00000001FF
